:020000040000FA
:1000000083168E100E141528A6000308A8000408F5
:10001000A7000A08A900612029088A00270884008F
:1000200028088300A60E260E0900FF2390009F01DA
:100030008312283085000730990083160830850028
:10004000D7308100960183128B012030840080011B
:10005000840A2A300402031D2728FC308100A030C6
:100060008B0000002830A100851932280A30A20038
:10007000A208031D3828851932280A30A200A208D8
:10008000031D3F28851932280A30A200A208031D4B
:100090004628A11A4F281B302502031D5328A3010F
:1000A000A401A501A00A5620A10034282008073980
:1000B000820709340A340C34183409340A340C34F5
:1000C00018340B1D0800FC3081000B11A20321081D
:1000D000A11A7228A30F6F28A40F6F28A50A22184F
:0800E0007228083085000800B9
:02400E00843FED
:00000001FF
